:020000020000FC
:10000000B3CD00000000000020C0AEC18EC00000D3
:10001000000098C000000000000000000203040679
:10002000080C10182030406080000406080C1018DE
:100030002030406080A0C0000003070F1F000D0D9E
:1000400004050D050305030302004FB662FD0CC055
:10005000552041F00994C52DC095089483FDC7959E
:10006000C4BD64604FBE1895C0916400089483FDC0
:10007000C795C4BD6B7FC0916400CF3F09F41EC01B
:1000800070FF1AC082FD05C04FBEC1989798959821
:10009000189576FD0EC065FD0CC0C091B100C0FD85
:1000A0009298C1FD9398C2FD9498CAEFC095CA95E5
:1000B000F1F7C198979895984FBE189524BCCC2716
:1000C000C064C8BF6460F8CFC6CF70FFC4CF65FD01
:1000D000C2CFC19AC0CF70FFBECF65FDBCCF979A8B
:1000E000BACF70FFB8CF65FDB6CF959AB4CF929ACC
:1000F00070FFB1CF65FDAFCFC7E0CA95F1F7C19AE8
:10010000AACF939A70FFA7CF65FDA5CFC7E0CA9588
:10011000F1F7979AA0CF949A70FF9DCF65FD9BCF82
:10012000C7E0CA95F1F7959A96CF4FB6C9B7CF7E7B
:10013000C9BF6E7FCCB5CE0DDDB5DF1DDBBDCABD41
:100140004FBE18953FB68F7EA9B7A072A2118061ED
:10015000A9B7AF7DA9BFA9B7AE7FA9BF7894A09179
:100160006800AA2341F085FD2BC0A0916800AA95E4
:10017000A093680025C040E050E085FD15C0A6B3FF
:1001800096FDA095A0FD4FEFAEB5A06496FDAF7BA8
:10019000AEBDAA27A062A8BF8D7FA6B396FDA0958D
:1001A000A0FD5FEF451739F7A8E161FDA093680056
:1001B00085FD03C0A8E1A09368004093960081608C
:1001C00085FD0EC0A0916900AA2331F0A0916900BD
:1001D000AA95A093690004C08061AA27A062A8BF65
:1001E00080FF3CC0A09196004A2F61FF8E7F85FD65
:1001F0001CC0A091B400A430C1F4403F08F040EF0F
:10020000A42FA295AF704A0F5091B600533069F0F9
:10021000A695A69550FD01C0A69552FD03C0A41B4E
:100220004A2F03C04A0F08F44FEF40936100A72FF5
:10023000A670A1F073FD12C0A0917000AA0FAA0FC2
:1002400050919E0056955695541708F0452F4A0F29
:100250004093610018F4AFEFA09361004091B400A7
:10026000443009F03EC0A0916100A093630040912A
:100270006300A0919B004A1708F04A2FA0919D00AF
:100280004A1708F04A2F542EA091A000AA2309F47F
:1002900022C0542F5A1B10F4A42F50E0BA2E889479
:1002A000AA1FAA2EA091A200A095AA22A50E58F0DE
:1002B000A091A100A21509F0AA95AA0EA093A100F1
:1002C00048F04A2D08C0A091A100BA1608F0A395E5
:1002D000A093A1004FEF409364007F7B485F08F03C
:1002E0007064A52DA03408F06860A0916000A3950B
:1002F000A093600059F0F894A9B7A160A9BF84FF4A
:1003000003C0A9B7A062A9BF3FBE1895A091740011
:10031000A395A093740041E050916800552329F003
:1003200085FF03C05A9550936800A0919600A130B4
:1003300018F0209299000DC020929A002092A300FC
:10034000A0919900AF5FA093990018F0AFEFA09330
:100350009900F894A9B7A160A9BF84FF03C0A9B709
:10036000A062A9BF3FBE18953FB646B557B58F7E70
:10037000A9B7A072A2118061A9B7AF7DA9BFA9B723
:10038000AE7FA9BF789481FD25C0AEB5AF7B96FD49
:10039000A064AEBD8260A6B396FDA095A0FF05C087
:1003A000409365005093660041C1AEB5A06496FDD0
:1003B000AF7BAEBDAA27A062A8BF8D7F85FF01C01D
:1003C00028C140E0A6B396FDA095A0FD22C14093B0
:1003D000960011C1AEB5A06496FDAF7BAEBD8D7F1A
:1003E00061FF72C0AEB5AF7B96FDA064AEBDAA271B
:1003F000A062A8BF82604093910050939200A090A9
:100400008F004A19B09090005B09BB24A22C4C3895
:10041000520518F42092950049C0A091D400AA2357
:1004200059F1483C520528F4A0E1BA2EAAE0AA2EC0
:1004300023C04836A1E05A0728F4A8E0BA2EAFE05E
:10044000AA2E1AC0403DA2E05A0728F4A4E0BA2E12
:10045000AEE1AA2E11C0403AA5E05A0728F4A2E066
:10046000BA2EACE3AA2E08C04839A8E05A0720F4F7
:10047000A1E0BA2EA8E7AA2EC42EA0919300CA1A12
:10048000D52EA0919400DA0ADD202AF4AFEFC094B3
:10049000D094CA1ADA0A20929500A8E0A210A0E02F
:1004A000CA14DA0618F4A1E0A093950040939300D3
:1004B00050939400409191005091920040938F008E
:1004C0005093900042E097C0A09165004A1BA09114
:1004D00066005A0B94FD82C093FD80C092FD7CC0E3
:1004E00086FF03C0D52EC42E0CC05695479591FDAE
:1004F00073C05695479590FD6FC0D52EC42ED694E7
:10050000C79461FD19C0AC2DAC51AD2DA24008F0CF
:1005100005C0DD2089F4AC2DA85C70F4A0916700C3
:10052000A395AA2311F0A0936700AA3008F471C024
:100530002092960081606DC0A0916700AA2319F0F7
:10054000AA95A0936700A22C5091BA0097FD06C00F
:10055000A090C800533011F4A090D000AAEFAA0ECA
:10056000A22DA21DCA18DA0A4FB74170533049F4C0
:10057000442321F087FD05C0806803C087FF01C0C8
:100580008F77442359F0533031F4AFEFC094D094B7
:10059000CA1ADA0A03C040E050E020C0533049F4E0
:1005A000CC0CDD1CAAE0CA1AD20818F4A0E0CA2EAE
:1005B000D22CAFEFCA16D20418F04FEF50E00EC0A5
:1005C000A091AC00CA9E412D000C441F50E008F0E1
:1005D00012C04FEF50E00FC05695479594FF07C0EB
:1005E000552309F04FEFA42FA6954A0F521D4F3FF8
:1005F000520508F04FEF40939600816061FF09C0FB
:10060000AFE1A095A923AB299A2F8F7DBB2009F4D8
:100610008062A8E1A093680085FF03C0AAE0A093D0
:10062000680061FD03C085FD01C08F7E85FD03C0AC
:10063000A6E0A0936900F894A9B7A160A9BF84FFC0
:1006400003C0A9B7A062A9BF3FBE189511E00AC0B8
:1006500013E008C01AE006C01EE104C014E602C0A0
:1006600018EC00C005E1BB27BA95F1F70A95D9F758
:100670001A95C1F708952AE338E709C020E33CE85A
:1006800006C02AE234EB03C025E238EC00C012E0D9
:10069000BB27939ABA95F1F7979ABA95F1F797987D
:1006A000BA95F1F79398BA95F1F7123009F0C19A1B
:1006B000123009F4959AB091AD00BA95F1F7123065
:1006C00009F0C198123009F49598B7E8BA95F1F796
:1006D0001A95F1F6022FB22FBA95F1F70A95D9F7CC
:1006E0003A95A9F6939A0895221B39E0001F3A958E
:1006F00009F40895221F211B18F4210F8894F6CFC6
:100700000894F4CF622C722CB0E08894B395221F29
:10071000331FE0F7379527958894912E802E020B92
:10072000130B10F4192D082D10F4889401C00894AF
:10073000661C771CBA9571F7172D062D0895322D7A
:1007400011232AF43A9500951095031B130BF89486
:10075000029F712C002D129F912C802C7894780C84
:10076000172D921C292DB4E06B2E26951795079511
:100770006A94D9F7332321F000951095031B130BCE
:1007800008950091B4000430A1F1B0919600B150E9
:1007900008F010C0B0916100B093630020927E0019
:1007A00020927F002092800020928100209282007F
:1007B0006F7B1FC06090B4006064B0916100B09323
:1007C000620008E317EC20917A0030917B003695A7
:1007D0002795B62DBA9541F036952795B62DBA9541
:1007E000BA9511F0369527958DDF00937E00109312
:1007F0007F00089500917E00B09162000B1B109164
:100800007F00120928F40038BFEF1B0740F009C031
:100810000F37120508F405C00FE710E002C000E82A
:100820001FEF0093830010938400089500918300CC
:10083000B09180000B0F10918400B09181001B1FBC
:1008400020E03091840033230AF42A95B09182008D
:100850002B1F1AF4203F40F00AC02F3008F407C0C5
:100860000FEF1FEF2FE003C000E010E020EF30910A
:100870006300B0919B003B1718F4323030F009C090
:10088000B0918400BB235AF004C0B0918400BB2314
:1008900032F4009380001093810020938200089529
:1008A0002091D70000918300000F10918400111F48
:1008B00046DF11232AF40038BFEF1B0740F009C0C0
:1008C0000F37120508F405C00FE710E002C000E87A
:1008D0001FEF002352F0B0916200B01B0B2F18F0F5
:1008E000013008F00AC001E008C000950F5FB09128
:1008F00062000B0F08F001C00FEF00938500089510
:100900002091D800009181001091820018DF1123FE
:100910002AF40130BFEF1B0740F009C00F3F12055A
:1009200008F405C00FEF10E002C001E01FEF112333
:1009300052F0B0918500B01B0B2F18F0013008F079
:100940000AC001E008C000950F5FB09185000B0F51
:1009500008F001C00FEF0093630008950FEF677F69
:1009600071FD29C072FD09C06860B0917B00BA308A
:1009700020F0B52DB03408F4677FB091D300BB23CD
:10098000D1F0B0917B00BB23B1F00FEF10917B0051
:10099000ABDEF894B091730072FDB5E00B9F112DA2
:1009A000002D7894112309F00FEFB0919E000B17E2
:1009B00010F400919E0000939D00089500917A002C
:1009C00010917B0000541140B0919D0010F4BA9535
:1009D00001C0B39511F0B0939D00089500C0089533
:1009E0002091B500B6B1B6FDFBCF04B115B1B6B1DB
:1009F000BF77B6B9B091AA00B395B093AA00B8304A
:100A000060F12092AA00B091D200BB2321F1112302
:100A100029F0B091AB00BF3F61F009C0B091AB00CD
:100A20000B1739F020F4BB2321F0BA9502C0B3951F
:100A3000E1F300919B00B093AB00BA3F50F400EC9F
:100A4000B93F38F400E8B83F20F400E4B73F08F4B9
:100A500000E000939B007F7E089510919B00B0E121
:100A60001B0F08F41FEF10939B00B091B400B4303B
:100A700081F000919B00B0916300B01B10F40091D5
:100A80006300B0919D000B1708F00B2F502E0093C0
:100A90006400B091AA00B73009F47061089502E3D0
:100AA000F894B091D9000B9F012D000C001F789491
:100AB000B0919B000B1710F000919B000093610018
:100AC00000936300502E0093640000939E000895ED
:100AD00020927A00B0EFB0937B000895F8940CB5A3
:100AE0001DB5209174007894309175006090760067
:100AF0000093750010937600031B160971FD03C067
:100B000077FD7DC027C0709077002093770027097C
:100B1000222311F00FEF1FEF809078009090790062
:100B20003093780060927900009175001091760002
:100B30000819190920917A0030917B003695279584
:100B4000020F131F10F40FEF1FEF00937A001093A2
:100B50007B0029C020917A0030917B003901B4E0FC
:100B60008B2EB2E09B2E343010F08A949A94383059
:100B700010F08A949A94769467948A94E1F72619EF
:100B80003709992021F0169507959A94E1F7200FDF
:100B9000311F20937A0030937B0028F43FEF30938D
:100BA0007A0030937B00323008F4706871FF02C025
:100BB000B3E00DC0B091C40000917100023838F06C
:100BC000B395003A08F0B395B63008F0B5E09B2E27
:100BD000B4E08B2E10917B0000917A0024E01695F2
:100BE00007952A95E1F70819120928F0B02FB2509D
:100BF000B12FB20910F402E010E0980126C0209154
:100C00007A0030917B0039017694679466946694FB
:100C100066942619320906950695200F321D2093F9
:100C20007A0030937B00323008F07F7704E036950D
:100C300027953695279526952695201B10F022306E
:100C400008F422E089019090C40060FDFECFE0909E
:100C50008B00F0908C006160B9B7B061B9BF38010A
:100C600077FD41C07694679400938B0010938C00BD
:100C7000B92DB330E1F0B0FD04C0060D171D93018E
:100C800006C0000F111F0250120922E030E0B92DFA
:100C9000B33068F020938D0030938E00009387006E
:100CA000109388006092890070928A003AC0009385
:100CB0008D0010938E0020938700309388006092FF
:100CC000890070928A0071FF0DC0BFE0B0938D0063
:100CD00020928E00B093890020928A00B0938B00FE
:100CE00020928C001EC0669400938B00B92DB33007
:100CF00091F0B0FD03C0060D262D03C0000F025079
:100D000022E0B92DB33038F020938D000093870096
:100D10006092890006C000938D0020938700609246
:100D2000890000917C0002FD0350013029F495FDFB
:100D30000AC0B0E0B7B909C0023019F4B7E0B7B9DA
:100D400004C095FDF6CFB6E0B7B90091A200000F40
:100D500010F4BBE60B270093A20060FDFECFB2E0CB
:100D6000B0936E006160B9B7B061B9BFB72FB6700C
:100D7000D1F020917A0030917B00369527953695F9
:100D8000279571FF02C0B0E43B0FF8940CB51DB578
:100D9000020F131F1BBD0ABD6160B0E1B8BFB9B738
:100DA000B061B9BF78940895606120927D0020E021
:100DB00067FD20E206C0606120927D0020E267FDB1
:100DC00020E001E011E077FD11C0B72FB67009F007
:100DD0006F7E14E100917B00069509F403950F30B6
:100DE00008F00FE071FF02C004E114E160FD0FC0E4
:100DF000B0917D00BB2359F071FF06C0B0916E0029
:100E0000BA95B0936E0011F4706247C0ABDFB0B713
:100E1000B77FB0BFB8B1B0B7B860B0BFB0917D0018
:100E2000B395B0937D00B8B177FD06C0B1E071FD18
:100E3000B3E0BA95F1F7B8B1B072B21709F022C0B9
:100E400071FF05C00395011708F00A95CFCF64FD27
:100E500005C00395011708F0B4CFC8CF6F7EF89492
:100E60003CB56DB470907A0080907B00370D681CA3
:100E70006BBC3ABD6160B0E1B8BFB9B7B061B9BF92
:100E800078949FCFB0916D00B13008F49ACF64FD93
:100E900098CF0A9509F0AACF7F7D20918D003091DF
:100EA0008E00F894B0E1B8BF0CB51DB5020F131F4A
:100EB0001BBD0ABDE0908700F09088006160B9B763
:100EC000B061B9BF7894B72FB67039F0B0916D00AA
:100ED00072FFB395B0936D0009C075FF07C067FD41
:100EE00005C064FD03C0BF91BF91EEC4089500E04A
:100EF00063FF03C064FF01C001E0F894109171002A
:100F0000B7E01B9F212D102D7894200F2695179563
:100F1000269517952695179510937100183718F494
:100F2000B8E7B093710000917100B09172000B1797
:100F300020F06062C1989798959860FDFECFE09090
:100F40008900F0908A006160B9B7B061B9BF0895B7
:100F5000B2E095FD0AC0F894B0937C00939A929801
:100F600062FF01C0959A7894F4C0F894B0937C0025
:100F7000939A949862FF01C0C19A7894EAC0B3E052
:100F800082FF24C095FD11C002E0F894B0937C006C
:100F9000E1E8F0E00093B1009598949A62FF02C0F6
:100FA000979A01C093987894D4C002E0F894B093D3
:100FB0007C00E1E8F0E00093B100C198929A62FFF2
:100FC00002C0979A01C093987894C3C095FD0BC056
:100FD000F894B0937C00EBE6F0E0959862FF01C0D6
:100FE000979A7894B6C0F894B0937C00EBE6F0E062
:100FF000C19862FF01C0979A7894ABC0B4E095FDA8
:101000000AC0F894B0937C00929A949862FF01C051
:10101000979A78949EC0F894B0937C00949A929892
:1010200062FF01C0979A789494C0B5E082FF24C013
:1010300095FD11C001E0F894B0937C00E7E7F0E083
:101040000093B1009798939A62FF02C0C19A01C0C1
:10105000929878947EC004E0F894B0937C00EBE81A
:10106000F0E00093B1009798939A62FF02C0959ABE
:1010700001C0949878946DC095FD0BC0F894B0931E
:101080007C00E5E6F0E0979862FF01C0C19A789491
:1010900060C0F894B0937C00E1E7F0E0979862FFBD
:1010A00001C0959A789455C0B6E095FD0AC0F894B1
:1010B000B0937C00949A939862FF01C0C19A78948F
:1010C00048C0F894B0937C00929A939862FF01C054
:1010D000959A78943EC0B1E082FF24C095FD11C07E
:1010E00004E0F894B0937C00EBE8F0E00093B100EA
:1010F000C198929A62FF02C0959A01C09498789420
:1011000028C001E0F894B0937C00E7E7F0E000939A
:10111000B1009598949A62FF02C0C19A01C092985A
:10112000789417C095FD0BC0F894B0937C00E1E76C
:10113000F0E0C19862FF01C0959A78940AC0F894D3
:10114000B0937C00E5E6F0E0959862FF01C0C19A9B
:1011500078946F7D089524E630E0F9012092B10083
:10116000C19897989598929A939A949A6B7F0895BC
:10117000A2EBB0E009E00D9309E00D9304E00D93BC
:101180000FEF0D9303E00D930FEF0D9309E00D9317
:1011900003E00D9301E00D9301E00D93AEEBB0E0A1
:1011A00001E00D930FEF0D930D930D930D930D93A0
:1011B00003E00D930FEF0D930FEF0D930D9305E2E9
:1011C0000D9300ED0D9308E20D9300E50D9304E0FF
:1011D0000D930FEF0D9302E00D9300E00D930AE7DE
:1011E0000D930FEF0D9300E00D9301E00D9300E0E0
:1011F0000D9303E00D9300E00D9308952091B90045
:101200008B7F233009F48460B091BA00B33019F0B9
:101210009F7DB1FD90629F7BB091BB00B1FD90645A
:10122000223011F0886001C0877F08950A95E00F91
:10123000F21DB4910895ECE1F0E00091B200F6DF08
:10124000B093D700ECE1F0E00091B300EFDFB09392
:10125000D800EAE2F0E00091B800E8DFB093D900EE
:101260000091B800023008F402E000937300B091DE
:10127000CE000FEFB23009F400EAB33009F402E80F
:1012800000937200E8E3F0E00091D500CFDFB09367
:10129000A000089508952091C8003091C900B09130
:1012A000BA00B33009F43E5097FF02C020E03FEF90
:1012B000B32FB21B6B2EB25810F4B2E86B2E00E0C5
:1012C0000395609EB12DBD57D8F30093AC000895EF
:1012D0009068E1DFC1D920E030E0B0E16B2EB8D9F1
:1012E000B09196002B0F321D6A94C9F7B4E0369581
:1012F0002795BA95E1F7822E9F77CDDF0895F89470
:10130000E3E0F0E0B9E0B7BFB491B078C1F3F8948E
:10131000A895B1B5B861B1BDB0E0B1BDB4E0BEBF94
:10132000BFE5BDBF18DFB0E0B8BBB2E1B7BBB0E00E
:10133000B5BBB0E0B4BBBCE1B2BBBCEBB1BB2224DB
:10134000A0E0B0E02D92AA31E9F7A0E6B0E00FEFFF
:101350002D920A95E9F7B1E0B093A20009DFECD233
:10136000B6B1B460B6B90091CA000093AD00B1E067
:10137000B0936A00F89474D97ED96ED97FD96CD9AC
:1013800080D96AD9F8940AEF1AEFA6B396FDA09512
:10139000A0FF1FC01A95C9F70A95B1F7E0E0FCE17C
:1013A000B591B43E39F4B591B03E21F4B591BF3F4B
:1013B00009F40CC0E0E0F395F395B591B83F49F41A
:1013C000B591B43931F4B591BA3A19F4EE27F695DE
:1013D000099414DF30DF5EDF5EDF0091CA00009306
:1013E000AD00B9DEB2E0B3BFB2E0BEBDB2E0B5BDA4
:1013F000B1E5B8BFB9BFB0B7B77FB0BFB8B1B0B78C
:10140000B860B0BF23D97894E9DA20927000BEB5F5
:10141000B06496FDBF7BBEBDB9B7B062B9BFBB2794
:10142000B062B8BF8D7F1CD9626033E02CE0B09110
:101430009500BB2321F42CE03A9509F4A3CF0CD9F5
:1014400080FFA0CF8E7FB0919600B23078F3B92F95
:10145000BF710091980000939700B0939800B01767
:1014600029F72A9521F76D7FBEB5B06496FDBF7B45
:10147000BEBDBB27B062B8BF8D7FB091D400BB2387
:1014800021F48062B92FB0709B2F8F7B2092670070
:10149000E5D885FF05C0B0916700BA3008F08064D8
:1014A000D7D802E085FF01C000E0B0919600B017E8
:1014B000B8F3F894E0D8DFD8DED87894D1D8209269
:1014C0008600B091BA00B33009F473C0C1D8B091AE
:1014D000BE00B13008F46DC0B0916A00B13008F4BC
:1014E00068C085FD18C0B0919600BF3F08F461C088
:1014F000F894CAD87894B2D8B0919600B130C0F7B9
:10150000F894B9D8A7D8B7D87894A8D8B09196004D
:10151000BF3FB0F3D2C2B3E09B2E9068F894BBDE1D
:1015200078949CD8F8949F77B6DE80909600B0911E
:101530009600BF37789408F444C088D8F894A4D8AB
:1015400078949A9451F7C4DEB82DB093C90088D826
:10155000F8941FD285D27894BAE09B2E9068F894C4
:101560009ADE78947BD8F8949F7795DE80909600E9
:10157000B0919600BF37789478F768D8F8947BD804
:1015800069D879D878949A9449F7A2DEB82DBB5FD0
:10159000B093C80065D8F894FCD171D278945ED825
:1015A000F89479DE7894B0919600BF3F08F499CF13
:1015B00084C200919600B09186000B1710F0009342
:1015C00086004CD801E0B091BA00B35009F405E0B0
:1015D000B0919600B01708F074CFF89455D854D84D
:1015E00053D878943DD820926A0020926B002092C4
:1015F0006C00B0916B00B395B0936B00BF3F71F579
:10160000B0916C00B395B0936C00B091CC0009E13F
:10161000BA9559F002E3BA9541F00DE7BA9529F071
:101620000AEFBA9511F020926C00B0916C00B017DF
:10163000A8F091DD0BD8B0916C00BA95B0936C0016
:1016400020926B00B091CB00B093AD00F8941CD801
:101650007894B091CA00B093AD0000D8FBD7B09198
:101660006800BB2319F485FF01C08CCE01E085FD25
:1016700001C006E0B0919600B01708F4BACFB0915F
:10168000BA00B35009F0EAD7B0916800BB2309F45F
:1016900079CEF89460DD2092610020926200209261
:1016A0006300522C209264002092A1007894B091A3
:1016B000B700BB0FB0939F0020927E0020927F0066
:1016C0002092800020928100209282002092AA0025
:1016D00060E070E020927100B8E0B093AA00706101
:1016E000B5D7B2E074FDB1E0B7B9B6B1B068B064D7
:1016F000B6B9B6B1B6FDFDCF04B115B1B6B1BF777D
:10170000B6B9112309F00FEF0093AB0069D9B8E027
:10171000B093AA00706172DDF894BFEFB0939B00A4
:10172000BED9B0916100B0939B00B0939C00B09380
:101730009D007894B1E0B0936100B09363005B2E9C
:10174000B0936400B093A400B0919A00B093A3004A
:10175000B091BA00B33019F49F7D87FD906271603B
:10176000726020926D00A0DCB6DCB2D9B7D9B0D9D6
:10177000B5D9AED920DB05D8BADBEADBAFD914DBAB
:1017800066FD38D877FFEAD877FD18D9B0DBF7DBEC
:10179000A5D911DB66FD4AD8AADB30DC9FD904DB72
:1017A00066FD7ED8A4DB41DC99D905DB66FDA8D8AF
:1017B0009EDB7ADC93D9F8DAB2E074FDB1E0B7B918
:1017C000B6B1B068B064B6B992DB85DC87D908D908
:1017D00071FF24C0B0919E00B0939B00B0939C0019
:1017E000B0919A00B093A300B1E0B093A40018E1C7
:1017F0002CE0B0916D00B11758F07D7F746020939C
:101800006F00B0919E00B0939B00B0939D0006C006
:10181000B0919600B13008F0ADCF60C072FF11C03A
:1018200067FD0FC0B0916F00BA9519F47B7F7860A7
:10183000A1CFB0936F00B0919600B13008F09ACF6D
:101840004DC020927000B09199000AEF1091D6001F
:10185000112309F003E0B01708F040C085FF04C071
:10186000B0916800BB23D1F1B091BA00B33081F4DC
:1018700095FD03C087FD04C00BC087FF01C008C0F1
:1018800067FD06C06068B0919E00B0939B0087CF53
:1018900000EF67FF05C0B0919E00B0939B0000E28F
:1018A000B0917B00B01708F465CF67FF17C06F7762
:1018B0009F7D87FD90627460B2E1B0936F00B0913C
:1018C0009E00B0939B0056CFB0917000B395B0933B
:1018D0007000B0919600BB2309F002C02092700006
:1018E000F89439DC8090B900B2E0B093B90086DC9E
:1018F0008092B900209261002092620020926300E1
:10190000522C2092640020929F0060E070E0789456
:10191000A5D621DC0091D600002319F0C19A979A30
:10192000959AB6B1B460B6B985FF05C0B0917000A4
:10193000B43008F027CD59CEEDE0F0E023D00535E6
:1019400009F01BC0EEE0F0E01DD00A3A09F015C026
:101950003AE0A2EBB0E0E3E0F0E014D00D93319672
:101960003A95D9F739E1AEEBB0E0EFE0F0E00AD01C
:101970000D9331963A95D9F702C0FADB0AD0E8E226
:10198000F0E00895E199FECFEEBBFFBBE09A0DB306
:1019900008951ED03AE0A2EBB0E0E3E0F0E00D9154
:1019A0000FD031963A95D9F739E1AEEBB0E0EFE0E0
:1019B000F0E00D9105D031963A95D9F712D00895FF
:1019C000E199FECF0DBBEEBBFFBBE29AE19A089511
:1019D000EDE0F0E00FEFF4DFEEE0F0E00FEFF0DF2E
:1019E0000895EDE0F0E005E5EBDFEEE0F0E00AEA77
:1019F000E7DF08953091AE000091AF00313011F46F
:101A00000093B200323011F40093B300333011F47C
:101A10000093B400343011F40093B600353011F463
:101A20000093B800363011F40093C400373011F43D
:101A30000093B900383011F40093D500393011F417
:101A40000093CE003A3011F40093BA003B3011F409
:101A50000093BB00089525E003D62A95E9F7089581
:101A60000AD60CD60ED610D6F5D505D607D609D689
:101A70000BD6F0D500D602D604D606D6089504D6E5
:101A800000D6FCD5F8D5E6D5FFD5FBD5F7D5F3D5EF
:101A9000E1D5FAD5F6D5F2D5EED508958090AE0011
:101AA0009090AF00E8D5E7D5E6D5D4D58A94D1F7A4
:101AB000EBD5D0D59A94E1F70895F894D1DF7894D6
:101AC000CADFC9DFB1E0B093AE00B1E0B093AF00C0
:101AD0002092B000F894E2DF7894B5E06B2E70901D
:101AE0009600BED5B09196007B16C9F7B13018F0BC
:101AF000BF3F40F107C07EDFF8944BDFB1DFB8E0B5
:101B0000B1BDA9DF6A9459F7B091B000B395B09315
:101B1000B000B33008F4DECF9EDFB091AF00B395D4
:101B2000B093AF00F894B091AE00BA95EEE3F0E058
:101B3000EB0FF21D049178940395B091AF00B017AC
:101B400008F4C6CF88DF87DFB091AE00B395B093BD
:101B5000AE00B091AE00BC3008F4B7CF09DBF8940A
:0A1B600018DFB8E0B1BD77DFCACB93
:00000001FF
